:020000040000FA
:0600000016EF01F01200F2
:06002A0001004402000089
:08003000600000001000000058
:08003800D9CFE6FFE1CFD9FFAB
:10004000E652DF6ADFCF04F0FE0EDB50E76E0418E5
:10005000E8AE02D0E73402D0E750045C07E2100EAD
:10006000E66EFFEC00F0E552DF2AECD7E552E552F0
:10007000E7CFD9FF1200816A806A0F0EC16E1F0E92
:10008000926E936A80A808D08050816E010EE66E51
:10009000FFEC00F0E55262D0816A050EE66ECCDF1F
:1000A000E55200017A6B080EE76E7A19E8AE02D0CD
:1000B000E73402D0E7507A5D13E280B811D0010E28
:1000C0007AC0E7FFE75204E0E846FE0BE706FCE1F2
:1000D000816E050EE66EB0DFE55200017A2BE3D7A4
:1000E0007A6B080EE76E7A19E8AE02D0E73402D0D8
:1000F000E7507A5D14E280B812D07A29046E010EBE
:10010000045204E0E846FE0B0406FCE1FF0F816E9A
:10011000050EE66E91DFE55200017A2BE2D77A6B8D
:10012000100EE76E7A19E8AE02D0E73402D0E7503D
:100130007A5D14E280B812D07AC0E9FFEA6AE9BEBB
:10014000EA68600EE926000EEA22EF50816E050E85
:10015000E66E72DFE55200017A2BE2D793D71200E8
:100160002A0EF66E000EF76E000EF86E0001090002
:10017000F550756F0900F550766F03E1756701D092
:100180003DD00900F550706F0900F550716F0900FE
:10019000F550726F09000900F550E96E0900F5503D
:1001A000EA6E090009000900F550736F0900F55067
:1001B000746F09000900F6CF77F0F7CF78F0F8CF29
:1001C00079F070C0F6FF71C0F7FF72C0F8FF000150
:1001D000735302E1745307E00900F550EE6E7307A4
:1001E000F8E27407F9D777C0F6FF78C0F7FF79C057
:0E01F000F8FF00017507000E765BBFD7120006
:0201FE00FF0EF2
:10020000E350036EEF0E01D0F30EE76EE72E06EF1C
:1002100001F00C0E026EE76AE72E0CEF01F0022EE1
:0C0220000BEF01F0032E04EF01F01200C0
:04022C0013EE00F0DD
:1002300023EE00F0F86A019CB0EC00F03BEC00F01B
:04024000FDD71200D4
:0C0244003F065B4F666D7D077F6F777C87
:04025000395E797129
:020000040030CA
:0E000000100F1F1E008181000FC00FE00F4087
:00000001FF
